:0D0059005391DF8FB2E59130E5FBAFB2228D
:10004300D2A530A5FDC2A37F24120059E4FF1200FC
:0500530059D2A3C2A573
:010058002285
:0C006600C2A4120043EFC313F58080F623
:10000300E4F595F594F5B475B302C2A37F0312002A
:10001300597F011200597F01120059D2A3C2A37F55
:1000230011120059E4FF120059EF54F1FED2A3C29A
:0F003300A37F01120059EE4402FF120059D2A31D
:01004200229B
:06007E00120003020066FF
:0300000002007289
:0C007200787FE4F6D8FD75810702007E5F
:00000001FF
